:020000040000FA
:10000000012807309F00850186018316FE30850098
:10001000FB3086001930990024309800831290300C
:1000200098006E20A101A1018C1A64206430210681
:100030000319452013288207533465346E34733412
:100040006F3472342034503449344E3447342934B8
:10005000293429342C34203452346F3462346F34D0
:1000600074347334203441347234673465346E34FC
:10007000743469346E3461342C3420343234303486
:10008000303438340D340A340034A0010514000033
:10009000000000000510831605148312A201A203BC
:1000A000031D4F28A301A20A0319A30A0518532808
:1000B0008316051083123D30682020306820230805
:1000C0007B2022087B2077281A08A10068200800DE
:1000D00099008316981C6A2883120800A001200842
:1000E0001B20003E031908006820A00A6F280D306D
:1000F00068200A306828A700270E81202708812061
:1001000008000F39A400093C031889282408373E49
:0801100068282408303E68282D
:02400E00503F21
:00000001FF
